:020000040800F2
:1000000000200020852000082D1D00082F1D00085D
:1000100000000000000000000000000000000000E0
:10002000000000000000000000000000311D00087A
:100030000000000000000000331D0008351D00080E
:10004000D520000800000000D5200008D5200008B9
:10005000D5200008D5200008411D00084B1D0008D0
:1000600000000000551D0008651D0008D52000088F
:10007000D5200008D5200008D52000080000000089
:10008000D52000080000000000000000D520000876
:1000900000000000D5200008D5200008D520000869
:1000A000D5200008D5200008D52000087D1D0008B7
:0800B000D5200008000000004B
:1000B80010B5064C2378002B07D1054B002B02D036
:1000C800044800E000BF0123237010BD8000002019
:1000D80000000000F8660008044B10B5002B03D0A0
:1000E8000349044800E000BF10BDC04600000000FE
:1000F80084000020F86600080023C25C0133002A4F
:10010800FBD1581E7047000002B4714649084900E7
:10011800095C49008E4402BC7047C046002243086F
:100128008B4274D303098B425FD3030A8B4244D3B7
:10013800030B8B4228D3030C8B420DD3FF220902F9
:1001480012BA030C8B4202D31212090265D0030BB8
:100158008B4219D300E0090AC30B8B4201D3CB03AE
:10016800C01A5241830B8B4201D38B03C01A5241F0
:10017800430B8B4201D34B03C01A5241030B8B42F2
:1001880001D30B03C01A5241C30A8B4201D3CB02DD
:10019800C01A5241830A8B4201D38B02C01A5241C2
:1001A800430A8B4201D34B02C01A5241030A8B42C5
:1001B80001D30B02C01A5241CDD2C3098B4201D3DD
:1001C800CB01C01A524183098B4201D38B01C01A5B
:1001D800524143098B4201D34B01C01A52410309D2
:1001E8008B4201D30B01C01A5241C3088B4201D381
:1001F800CB00C01A524183088B4201D38B00C01A2E
:10020800524143088B4201D34B00C01A5241411A54
:1002180000D20146524110467047FFE701B5002061
:1002280000F0F0F802BDC0460029F7D076E7704725
:1002380003460B437FD4002243088B4274D303093F
:100248008B425FD3030A8B4244D3030B8B4228D3E0
:10025800030C8B420DD3FF22090212BA030C8B4206
:1002680002D31212090265D0030B8B4219D300E0A6
:10027800090AC30B8B4201D3CB03C01A5241830B2B
:100288008B4201D38B03C01A5241430B8B4201D3DB
:100298004B03C01A5241030B8B4201D30B03C01A04
:1002A8005241C30A8B4201D3CB02C01A5241830A7E
:1002B8008B4201D38B02C01A5241430A8B4201D3AD
:1002C8004B02C01A5241030A8B4201D30B02C01AD7
:1002D8005241CDD2C3098B4201D3CB01C01A52413E
:1002E80083098B4201D38B01C01A524143098B42C7
:1002F80001D34B01C01A524103098B4201D30B01B0
:10030800C01A5241C3088B4201D3CB00C01A5241D4
:1003180083088B4201D38B00C01A524143088B4299
:1003280001D34B00C01A5241411A00D20146524132
:10033800104670475DE0CA0F00D04942031000D351
:100348004042534000229C4603098B422DD3030AA6
:100358008B4212D3FC22890112BA030A8B420CD3B6
:10036800890192118B4208D3890192118B4204D3DF
:1003780089013AD0921100E08909C3098B4201D35F
:10038800CB01C01A524183098B4201D38B01C01A99
:10039800524143098B4201D34B01C01A5241030910
:1003A8008B4201D30B01C01A5241C3088B4201D3BF
:1003B800CB00C01A524183088B4201D38B00C01A6C
:1003C8005241D9D243088B4201D34B00C01A524143
:1003D800411A00D20146634652415B10104601D3D0
:1003E8004042002B00D54942704763465B1000D35A
:1003F800404201B5002000F005F802BD0029F8D000
:1004080016E770477047C0469E2110B5C905041C01
:1004180001F0D2F9002803D1201C00F0EFFA10BD3A
:100428009E21201CC90500F045F900F0E7FA802359
:100438001B069C466044F2E7F0B54F464646D64652
:1004480043025B0A4500C0B599460F1C2D0EC60F26
:10045800002D00D188E0FF2D00D18DE08022DB0047
:10046800D2041A430023914698469A467F3D7C025F
:100478007B00640A1B0EFF0F002B68D0FF2B21D0D6
:100488008022E400D204144342467F3B5B190021DA
:100498005D1C0A2A2EDC7E404246022A23DC013AF1
:1004A800012A00D9BDE002296ED001292CD10020F3
:1004B8000022C005F60710433043E0BCBA46B146F7
:1004C800A846F0BD2B00FF33002C65D0032241461F
:1004D80011433200013588467A40FF350A2900DD8C
:1004E800D8E016000321404601228240A620C00021
:1004F800024220D05346022B46D0032B00D1BBE04A
:1005080051464C460129D2D02B007F33002B70DD99
:10051800620704D00F222240042A00D004342201AA
:1005280003D5634B1C402B008033FE2B2CDCA2012F
:10053800520AD8B2BDE790208000024227D1B938CC
:10054800FF3810426DD03E00A1468A46D2E7002C03
:1005580041D1012342461A4390462B0042460121CD
:100568005D1C0A2A97DDC5E7002B26D1042398468F
:10057800033B00259A467AE7002B18D108239846B2
:10058800063BFF259A4672E7FF20002291E780226A
:100598000026FF20D2038CE7414602220135114391
:1005A8008846FF350A29A5DC02217E4074E70C2322
:1005B8009846093BFF259A4659E7180001F006F9C5
:1005C8004A46431F76259A4000236D429146984635
:1005D8009A462D1A4BE7200001F0F8F84246431FCF
:1005E8009C402B1A763B00215D1C0A2A00DC52E74E
:1005F80080E70122D31A1B2B00DD58E79E35220025
:10060800AC40DA40631E9C412243530704D00F23B9
:100618001340042B00D00432530137D501200022A7
:1006280047E7210C4A462404240C2700100C120426
:10063800120C44435743484351433A0C0919521882
:10064800944203D9802149028C4660443F04110436
:100658003F0CC9198C01671EBC41120C890E121877
:100668000C439201144312010ED5012362081C4069
:10067800144349E73E00A14680224B46D2031A4361
:100688005202FF20520A14E71D003DE792010020A4
:10069800520A0EE70F29EDD180224B46D2031342AE
:1006A800EAD01442E8D13E00FF20224301E7C046C9
:1006B800FFFFFFF7F8B54746CE464E024302450016
:1006C800720AC40F480080B594465F0A2D0E9B0934
:1006D800000EC90FB609FF2824D0012251402A1A5A
:1006E8008C420FD0002A00DC6AE1002835D1002EA8
:1006F80000D1A2E0511E012A00D124E1FF2A21D015
:100708000A002FE0002A00DC67E100285ED0FF2DF8
:1007180018D08021C9040E431B2A00DC76E02A0089
:10072800013332E02A00FF3A9146002E42D08C4233
:1007380055D04A46002A00D19CE0002D00D177E030
:100748000C003300DB08002B00D16EE08022D203BE
:1007580013435B02FF205B0A24E0FF2DF2D08021C7
:10076800C9040E4301211B2A08DC31002020D14096
:10077800821A96403200501E824111435B1A5A0178
:1007880060D407212A00194057D00F2119400429A5
:1007980000D00433590150D5501CFE2A45D09B0186
:1007A800C0B25B0AC0051843E4072043C0BCB94681
:1007B800B046F8BD012251408C42BAD14A46002ABF
:1007C80010D0002D00D198E00023BBE7002E34D0D4
:1007D800511E012A6ED0FF2AB4D00A009CE7002AD5
:1007E80000D088E0FE206A1C104200D092E0002D64
:1007F80000D0A4E0002B00D1CBE0002E00D0CAE04E
:100808000022DB085B025B0AD0B2CBE73100202074
:10081800D140821A96403200501E82410A439B18EA
:100828005A01AED56A1CFE2D4AD1FF200023B9E734
:10083800FF22002B4BD10C003300DB08FF2A00D12C
:1008480081E7DFE79F01BF09380000F0BFFF0538E7
:100858008740854221DC3B002021421B0132D340E6
:100868008A1A97407A1E974100223B43590700D0C5
:100878008BE78FE7FE206A1C104212D1002D52D15F
:10088800002B7CD0002EBBD09A1B500100D48BE0EB
:1008980001240022F31A0C40E8E7564B2A1A3B4081
:1008A800E4E79F1B7A0146D4002FCDD10024002015
:1008B800002377E79B1901250132590100D460E72D
:1008C80001214D4819405B0803400B43CEE7571EF2
:1008D800012A5AD00C00FF2A33D001221B2F07DC33
:1008E8002021C91B1A008B40FA40591E8B411A431C
:1008F8000500B31A43E7002D23D1FF22002B9BD01C
:10090800511E012AD6D0FF2A1BD01B292CDD02003C
:10091800731C3AE7FF2A88D09B195B08590700D057
:1009280033E7DB086EE7002B10D1002E43D00124FB
:1009380033000C4006E70124F71A0C4084E7002B2B
:1009480004D13300FEE601259B1B18E7002E00D1D9
:10095800F8E68022D203974204D3944502D20124B8
:1009680033000C40DB08F1E61A002025CA40691A5A
:100978008B40591E8B41134305009B1950E7002EED
:1009880094D0012433000C403AE70C000125F31AF7
:10099800F5E6330034E79B1900225901C1D5154A01
:1009A8001340DB0801222DE7002A00D17EE713005F
:1009B8000022DB0826E780230024FF20DB03F1E682
:1009C800002A00D156E7471B3A00002D00D130E736
:1009D8008022D2040C0013437FE7002A00D101E7EC
:1009E800411B002D01D10A0088E78022D20413435D
:1009F8008BE7C046FFFFFFFBFFFFFF7D4102420080
:100A0800C30F490A0020120E7E2A03DD9D2A02DD4B
:100A1800094A98187047802000040143952A07DC8A
:100A28009620821AD1404842002BF3D10800F1E702
:100A3800963A9140F7E7C046FFFFFF7F70B5041E66
:100A48000ED000F0C3FE9E2301001B1A962B0CDC6F
:100A580008282FD008398C406402640AD8B201E013
:100A680000200024C005204370BD992B16DC421FCE
:100A7800052800D09440220010480240650709D09C
:100A88000F252C40042C05D00432540102D59F2395
:100A980002405B1A9201540AD8B2E3E70200200030
:100AA8001B3290400200501E82410520401AC4406B
:100AB8001443E0E764029620640AD3E7FFFFFFFBD4
:100AC800F0B5DE46454657464E46E0B587B000923B
:100AD80001930B031B0B9B46CA0F4B000400804677
:100AE8005B0D029200D16AE1D44A934200D18CE1B5
:100AF8005946420FC9000A43802109041143C20024
:100B08009046CF4A894692469A440023002403938C
:100B1800009E019F3B031B0B9B467B0030005B0D37
:100B2800FD0F002B00D128E1C44A934200D177E1A0
:100B38005946720FC9000A438021090411438B46A4
:100B4800BF49F2008C4651466344CB1A9A460023AB
:100B5800029E6E400F2C27D8BA49A40009598F4627
:100B6800CB464246029E039B022B16D0032B00D194
:100B7800A6E2012B00D0DFE00022002300249046EB
:100B88001B052343F60733434046190007B0F0BC62
:100B9800BB46B246A946A046F0BD002200249046B6
:100BA800A64BEDE72E00DFE7CB4500D2D4E100D11C
:100BB800CFE101235B429C46444648460027E24475
:100BC8005B46150E1B021D43190C2B0412020095DF
:100BD8001D0C914602910395FFF726FB02006A431C
:100BE8000B04210C804619438A4209D9009D012330
:100BF800AC465B4261449C46E0448D4200D8FBE130
:100C0800881A0299FFF710FB039A24044243090447
:100C1800240C03000C43A24206D90099013B8C46E0
:100C28006444A14200D8E1E1A01A424612041A43E2
:100C380093464B4659461B0C1D0004930B0449462A
:100C48000904090C0C001B0C5C43120C6B4388460E
:100C580051436A43250CAC465B186344994203D957
:100C6800802149028C466244190C24041B04240C7C
:100C78008A181C19904202D316D1A74214D25B4697
:100C8800009D013B4F4405934F459B41AC465B4259
:100C98006344C018854200D3A1E1824200D9F6E13D
:100CA80000D1F1E1059B9B463C1BA742BF41009D3B
:100CB800801A7F42C01B854200D1D0E10299FFF71C
:100CC800B3FA039A0B044243210C070019438A42E2
:100CD80000D978E1881A0299FFF7A6FA039A240442
:100CE80042430904240C03000C43A24200D95DE1ED
:100CF8004146A41A3A041A43049D13041B0C594391
:100D080047466B439C46100C47430B0CBC4463445A
:100D180068439F4203D980256D02AC4660441F0C8E
:100D280009041B04090C3F185B18BC4200D202E1FD
:100D380000D1FDE001231A43434B5344002B00DC50
:100D4800AEE0510700D098E15946C90106D5594689
:100D58003E4B194080238B46DB0053443C498B4271
:100D680000DD1AE75946D208490711435A465B0580
:100D780054028846240B5B0D02E75A46009B1A432F
:100D880000D17EE05B46002B00D100E1584600F020
:100D98001DFD020003000B3A1D27009EBA1A190018
:100DA8005846D64008398840320002439346009A94
:100DB8008A40284953448A469A440023C8E65B4639
:100DC8000343994656D05B46002B00D1CDE05846E8
:100DD80000F0FCFC0B235B429C4602008444664600
:100DE8001D239B1B260011005846DE400839884009
:100DF80033000343994623008B409846164B002442
:100E08009B1A9A460023039382E65A460243914668
:100E18002AD100229A46022390460824039377E6B3
:100E28005A46009B1A430D4B9C46E244002A17D1B0
:100E380002231C4300239B46023389E6FF07000078
:100E480001FCFFFF20670008FF030000FFFFFFFE13
:100E5800FE070000F30300000DFCFFFF01F8FFFF91
:100E6800032332001C4373E69A460323D9460C2415
:100E780003934DE6002398469A46013304240393CE
:100E880046E601231C4300239B46013360E600230A
:100E9800802498460026924B240371E60122524290
:100EA8000121C91A382900DD66E61F2900DCABE0FC
:100EB8001F204042C31A5846D8400300202904D0B6
:100EC80058468849514488400243511E8A411A4372
:100ED800072319000024114013420CD00F2313409C
:100EE800042B00D1F9E0111D91429B410A005B429D
:100EF80059075B021C0BD2080A43904600233FE6C1
:100F080080244B462403234209D05B46234206D162
:100F18001C4324032E009046714B240B30E680249A
:100F28004B4624031C432403029E6D4B240B27E6E7
:100F3800002B00D100E70098511E84466444844287
:100F480000D284E0BC4200D2AEE000D1C1E00A0089
:100F5800F0E6424500D92CE64B46DC0758084346E4
:100F68005B081C434346DF072AE600F02FFC1523E5
:100F78009C4684440200634620321C2B00DC2EE78A
:100F880023000838834099460023984636E700F046
:100F98001DFC02000300153220331C2A00DCFBE68E
:100FA80000990838814000228B4602E70099013BEE
:100FB8008C466444A14200D99AE6A24200D897E63A
:100FC800831E644494E6AC466144013F8D4200D9D7
:100FD80080E68A4200D87DE6871E61447AE685422B
:100FE80000D05FE6B94500D95CE656E6A24200D8D3
:100FF8001AE6831E644417E68A4200D800E6AC4627
:10100800831E98466144FBE53748140050448240EB
:101018005B4617008340CC407A1E974123433B43ED
:101028001A005B46CB40510709D00F211140042913
:1010380005D0111D9142924152429B180A00190293
:1010480000D455E7002201230024904698E50A00C1
:10105800BC4200D06EE64B4500D06BE66CE6234BF5
:10106800234A5344924500DA18E7012149420A1DF0
:101078008A42894149428B4466E60F21114004297E
:1010880000D161E61100F2E7BC4200D80AE602236B
:101098005B429C4600994F444F459B41E3448C4634
:1010A8005B426344C018FFE54946009D4800484537
:1010B8008941AC46494261448146023A6418C7E70F
:1010C80080245B4624031C4324039046044B240BD2
:1010D80056E59945E8D30A00BDE7002308E7C0466E
:1010E800FF0700003E0400001E040000FF0300008C
:1010F80002FCFFFFF0B55746DE464E464546E0B5D2
:101108001F000B031B0B16009A46CA0F4B00040066
:10111800934687B05B0D00D1D5E0BB4A934200D11E
:10112800F8E05146420FC9000A43802109041143DF
:10113800C2009146B54A8A469D18002398460293F4
:101148003C037B00FA0F3000240B5B0D009200D1AA
:1011580096E0AD4A934231D0720FE40022438024D6
:1011680024041443A94AF000944663445B195A1CAA
:101178000192424600260A2A42DC5A4600994A4011
:1011880093464246022A32DC013A012A00D949E153
:10119800022E00D1CAE0012E3DD1002300240022F6
:1011A80010005A461B052343D2071343190007B002
:1011B800F0BCBB46B246A946A046F0BD924B2643BA
:1011C800EB18002E00D1BBE00322414611435A46DA
:1011D800884600994A40802109018C4629006144CB
:1011E800019141460A2900DD33E29346032642462F
:1011F80001279740A6213A00C9000A400F4231D082
:10120800029E022E00D135E2032E00D1D2E15446CF
:101218004846012EC1D0019A7D4B94466344002B69
:1012280000DCC0E0420709D00F220240042A05D0A2
:10123800021D82428041404224181000E20106D576
:10124800744B019A1C4080239446DB006344724A25
:1012580093426BDC6207C00864025B050243240BFF
:101268005B0D9DE7902189000F4263D188223A42A5
:1012780000D1D7E0009BA2469B4681460296BFE775
:101288002300334300D17FE0002C00D1ADE12000E2
:1012980000F09CFA020003000B3A1D201900821A84
:1012A80030000839D0408C400443300088405B4A05
:1012B800EB1A944663445A1C0192424600260A2AB5
:1012C80000DC5AE79CE753460343994654D05346FB
:1012D800002B00D177E1504600F078FA0B235B42EF
:1012E8009C460200844411005046083988401D235A
:1012F800804660461B1A2000D8400300404603433E
:101308009A4623008B4099460023444D9846AD1ACF
:10131800029315E752460243914626D100221D004A
:101328000223924608329046029309E700240022DD
:10133800354B35E7002380249B462403324B2FE7A7
:101348000222414611438022120194462A00624437
:10135800884601920A2900DD52E75A460020009982
:1013680004004A40934602260BE70C221D00032383
:10137800814690460293E3E600239A460433984652
:10138800033B00250293DBE6424601331A432B0058
:1013980090465A1C019242460024002001260A2A3F
:1013A80000DCEAE62CE70122D21A382A00DDF4E64E
:1013B8001F2A00DC2AE11F214942CB1A2100D9400B
:1013C8000B00202A05D0164A019D94466544AC407E
:1013D8002043421E9041184307231900002401406E
:1013E80003420CD00F230340042B00D140E1031D1E
:1013F8008342A4411800644261076402240BC208B6
:1014080000230A43CCE6C046FF07000001FCFFFFAB
:10141800FF030000FFFFFFFEFE0700000DFCFFFFBB
:101428003E04000049464A460904090C0D00160C02
:10143800020C0004000C4543AC4605007543A84661
:1014480015000F007543009202952A00009D6F4316
:1014580065462D0CA94647444F44B84505D91500A3
:10146800802252029046454402953D0C03956546FC
:101478002D043F042D0CAC463D0065440495250C15
:101488002404240CAC4625007543A84665460F0085
:101498006943414489466743390C49446E4388454A
:1014A80003D980225202904646440D0CA8463500C6
:1014B80045440595039D3F04A8463F0C0904C919F6
:1014C80088444546039555462E04360C2F0C3500A6
:1014D8004543784381463800A8462D0CAA46009A11
:1014E800504372434A445244914503D980256D02C2
:1014F800A9464844150CA94645462D042D0CA84676
:1015080065467D43120448449044A9463200654626
:1015180062436E437C43170C3619BF19BC4203D98A
:1015280080246402A446E144029C039EA446059DCF
:1015380066448E428941AC4612043C04120CA2183F
:101548006244494254184644A4464645A44182464A
:101558006442A046AA4292418C458941E244D04463
:10156800494252420A43A045A44182458941644206
:1015780049420C4341463F0CD2191219CC0D04992B
:1015880070020843411E884141464A44F60D520202
:101598003043490214430843D20135D50122430898
:1015A80002401343E0071843640834E6009BA24650
:1015B8009B4681468024534624031C4324034A4601
:1015C8002E4B240BECE500F001F915239C468444CE
:1015D8000200634620321C2B00DC84E60023994677
:1015E8002300083883409A468EE600F0EFF80200A0
:1015F8000300153220331C2A00DC4EE602003400BA
:10160800083A0020944052E6019304E61C4B21005E
:101618009C460300019DD3406544A940194303003B
:10162800AB40581E834119430800D4404B0709D0EA
:101638000F230B40042B05D00B1D8B4280414042E9
:1016480024181800230200D4D6E60123002400221F
:10165800A6E50F29AAD1802352461B031A42A9D016
:101668001C42A7D11C43009B02009B46034B97E5F5
:101678000024C1E60024014B220091E5FF07000089
:101688001E0400000B00020070B5164D0C0382B05A
:101698004900002000920193240B490DDE0FA94256
:1016A80004DD1148814203DD104BF01802B070BD13
:1016B8008020400320430E4C641A1F2C08DD0D4B7C
:1016C8005B1AD84003005842002EEFD11800EDE70E
:1016D800094B009A9C46030061448B40E240134347
:1016E800F1E7C046FE0300001D040000FFFFFF7F76
:1016F8003304000013040000EDFBFFFF70B5002861
:1017080016D0C317C5185D40C40F280000F05EF856
:10171800104B1B1A5B055B0D0A2814DC02002E0017
:10172800153296400B22121AD5402D032D0B03E0DB
:1017380000240023002500261B052B43E407234330
:101748003000190070BD0B3885402D0300262D0B85
:10175800F2E7C0461E040000844608006146FFE721
:101768001FB500F0C9F8002801D40021C8421FBDE8
:1017780010B500F049F84042013010BD10B500F036
:10178800BBF8002801DB002010BD012010BDC046B9
:1017980010B500F0B1F8002801DD002010BD0120CF
:1017A80010BDC04610B500F057F8002801DC002035
:1017B80010BD012010BDC04610B500F04DF800283E
:1017C80001DA002010BD012010BDC0461C210123F4
:1017D8001B04984201D3000C10391B0A984201D30C
:1017E800000A08391B09984201D30009043902A2EA
:1017F800105C40187047C046040302020101010151
:10180800000000000000000070B542004E024C00CD
:1018180045026D0A120EC30F760A240EC90FFF2A5D
:1018280010D0FF2C0CD00120A2420AD1B54208D119
:101838008B420FD0002A04D12800431E984100E0B3
:10184800012070BD0120FF2CFBD13543F9D14B405D
:101858001800F6E70020F4E730B5420044024D02D4
:10186800C30F4800640A120E6D0A000EC90FFF2A42
:1018780019D0FF280BD0002A1ED100280BD1002D2B
:1018880027D0002C34D100292FD0080030BD002DDE
:1018980028D1002A01D1002CF5D08B4207D1002B8A
:1018A80023D01800F2E7002C1CD1FF2814D0581EB2
:1018B800022318400138E9E70028F8D08B42F6D116
:1018C8008242F4DCEBDBAC42F1D80020AC42DDD242
:1018D800E5E7002CDAD0EAE7002D03D18B42E6D108
:1018E8000020D3E702204042D0E701204042CDE764
:1018F8008B42E8D0DBE7C04630B5420044024D02D7
:10190800C30F4800640A120E6D0A000EC90FFF2AA1
:101918001AD0FF280ED0002A1ED100280ED1002D83
:101928002AD0002C0CD08B421DD0581E0223184000
:10193800013810E0002D0DD1002A20D1002C1ED135
:10194800002923D0080006E0002C03D1FF28ECD1A1
:10195800002D17D0022030BD0028E6D08B42E4D1FC
:101968008242E2DC04DBAC42DFD80020AC42F2D297
:10197800002B0BD01800EEE7002CECD0D5E78B42FB
:10198800D3D1F5E700208B42E5D0CEE701204042D5
:10199800E1E7C0461FB50C22002101A804F071FE42
:1019A8008022184C184B12062261042223608023DF
:1019B8006261033A1B03A276E2612200636000239E
:1019C8002C32137007226263220020003C32A3608D
:1019D800E36023836362A36223631370E36400F00C
:1019E800C9FB002801D000F083F9084B20000193BF
:1019F800012301A9029300F025FD002801D000F081
:101A080077F91FBDF80000200024014002000004FF
:101A180070B505008EB01422002103A804F031FE31
:101A28001822002108A804F02CFE264B2A689A42A6
:101A380045D18023DB010893802308A81B060C935B
:101A480001F080FF002801D000F052F980211E4BE0
:101A580049031A6CA0200A431A641A6C00260A402B
:101A680001210192019A5A6BC0050A435A635B6BC4
:101A780005960B400293029B022303935B1803A96C
:101A8800049301F08BFA114C114B200023600523BD
:101A980063607B332361803363618023DB00A36150
:101AA8002023E36180235B01A660E660236200F0E7
:101AB800D7FFB04201D000F01BF92C65A5620EB02B
:101AC80070BDC04600240140001002409C00002068
:101AD8000800024007B501210C4B09209A6B0A4304
:101AE8009A639B6B00220B4001934918019B00F0FD
:101AF8001DFF092000F044FF002202210A2000F007
:101B080015FF0A2000F03CFF07BDC0460010024048
:101B1800F0B502270125A02689B01422002103A8C8
:101B280004F0AFFD394BF6055A6B30003A435A635F
:101B38005A6B37493A400192019A5A6B00242A435A
:101B48005A635B6B2A002B400293029B01F050FB07
:101B580030000022202101F04BFB2A0029002D48EB
:101B680001F046FB0423300003A903930495059470
:101B7800069401F013FA08230393C42330009B034F
:101B880003A90493059401F009FA2023300003A95E
:101B9800039304950594069701F000FA402330005A
:101BA80003A903930494059401F0F8F9802303939F
:101BB800882330005B0303A90493059401F0EEF930
:101BC80003A91448039504950594069401F0E6F9D1
:101BD800C0235B0103931123300003A904930594E8
:101BE800069701F0DBF922003900062000F09EFE7E
:101BF800062000F0C5FE22003900072000F096FEFE
:101C0800072000F0BDFE09B0F0BDC046001002403C
:101C180004180000000400500848094B10B5036080
:101C280003234360074BC360074B836001F002FB4B
:101C3800002801D000F05CF810BDC0465C0100200F
:101C480000300040FF0F0000B80B000010B592B044
:101C58003422002105A804F014FD1022002101A857
:101C680004F00FFD8020800001F01EFB0A2305937D
:101C7800F6330893002309930E9308330F93C02378
:101C8800DB0240221093802302240A929B053F3AEC
:101C980005A80B920C940D94119301F031FB0028C8
:101CA80001D072B6FEE7072303900490210001A833
:101CB8000193029401F084FD002801D072B6FEE77A
:101CC80012B010BD10B500F02BFAFFF7BFFF04F0FB
:101CD800D7FBFFF71DFFFFF7FDFEFFF75BFE00F0E8
:101CE800B7F800F0F1F8FFF797FF04F013F9FEE7F3
:101CF80072B6FEE701210A4B82B01A6C0A431A64D5
:101D08001A6C0A4080210092009ADA6B49050A434E
:101D1800DA63DB6B0B400193019B02B07047C0464E
:101D280000100240FEE7FEE77047704710B500F06C
:101D38000BFA04F0D7FB10BD10B5082001F066FAC5
:101D480010BD10B5802001F061FA10BD10B5024831
:101D580000F0E0FF10BDC0469C00002010B503480D
:101D680000F0D8FF024800F0D5FF10BD1402002093
:101D7800B801002070B5124C200002F049FB200089
:101D880002F08AFA102223680E4DD969114211D047
:101D98001A620D4A1378002B0CD10C4B0C481B68A7
:101DA800596820235B1ADBB2137012782900D2B26B
:101DB80004F094FC29002022200002F07DFF70BD71
:101DC80070020020E1050020010600201402002016
:101DD800A105002070470000084B026882B09A42B3
:101DE80009D18021064B09021A6C0A431A641B6C3C
:101DF8000B400193019B02B07047C0460020004091
:101E08000010024010B5040086B01422002101A879
:101E180004F037FC0C4B22689A4213D101210B4B7A
:101E2800A0205A6BC0050A435A635B6B0B400093B2
:101E3800009B102301930E3B029301A902330593E3
:101E480001F0ACF806B010BD0020004000100240C0
:101E580010B588B01C22002101A804F012FC174C10
:101E6800174B184A23600223636000232000A360F5
:101E7800E2602361A36101F09BFF002801D0FFF716
:101E880037FF200001F0BEFF002801D0FFF730FF28
:101E980060230193FA2300229B00200001A90293EA
:101EA8000392059202F014F8002801D0FFF720FFF2
:101EB8002000FFF7A7FF08B010BDC0466C01002046
:101EC80000200040E703000010B5184B184C0C2206
:101ED800236096239B01636000232000A360E360D6
:101EE80023616261A361E36123626362A36202F01A
:101EF80059FE002801D0FFF7FBFE0021200002F068
:101F080053FF002801D0FFF7F3FE0021200002F064
:101F18006BFF002801D0FFF7EBFE200002F026FF40
:101F2800002801D0FFF7E4FE10BDC046003801408C
:101F38007002002070B506008EB01422002103A89C
:101F480004F09FFB1822002108A804F09AFB334BE9
:101F580032689A4260D1012308A8089301F0F2FC84
:101F6800002801D0FFF7C4FE80212D4BC9011A6C4F
:101F780000250A431A641A6C2A480A400192019AF9
:101F88000222596B114359635B6B03A913400293F7
:101F9800029BC0230492039305950695079500F0CC
:101FA800FDFF214C214B20002360322363604E3318
:101FB800236180235B01A560E5606561A561E5613A
:101FC800236200F04DFDA84201D0FFF791FE331DBA
:101FD800DC67A662164B174C8022236033236360AC
:101FE800233BA3600023E3606361A361E361802373
:101FF80020005B012261236200F032FD002801D03D
:10200800FFF776FE1B2000220121F467A66200F08C
:102018008DFC1B2000F0B4FC0EB070BD00380140F0
:102028000010024000040050140200201C0002406E
:1020380030000240B80100200C4B026810B50400C3
:102048009A4212D10A4A0B49136C0B480B4013648D
:10205800C02101F055F8231DD86F00F05BFDE06F3B
:1020680000F058FD1B2000F097FC10BD003801401F
:1020780000100240FFBFFFFF000400500D488546D6
:10208800FFF7A8FE0C480D490D4A002302E0D4587A
:10209800C4500433C4188C42F9D30A4A0A4C0023AA
:1020A80001E013600432A242FBD304F0F3FAFFF715
:1020B80009FEFEE70020002000000020800000202C
:1020C800F8670008800000208C060020FEE700006A
:1020D80070B5104B05001978002901D1012070BD99
:1020E800FA208000FEF71AF80B4C01002068FEF772
:1020F80015F800F061FC041EF0D1032DEED80200A3
:1021080001202900404200F011FC044B20001D6012
:10211800E5E7C04604000020000000200800002079
:102128008023084A5B00116810B50B430320136035
:10213800FFF7CEFF041E03D1FFF7DCFD200010BD22
:102148000124FBE700200240034A044B11681B7876
:102158005B1813607047C046040300200400002089
:10216800014B18687047C046040300208068400788
:10217800C00F70470023F0B585B004000393984260
:1021880000D1F0E0856D9D4205D1FFF741FC2300A9
:102198005433E5651D70802325685B05AA681A42DB
:1021A80000D1A7E00022AB680192DB0008D410231D
:1021B8000126A26D01961343A365E36D3343E365DE
:1021C8002800FFF7D3FF1022A36D1340034300D06C
:1021D800CCE0A26D674B20691A400633FF331343E6
:1021E800A365AB68DB0761D4276BE1687B1E9F4161
:1021F800A368A27E0B43217E3F0389030B43617EC4
:10220800C9030B4351030B439C46002800DB86E0BF
:1022180041004908230066462C331B785B00334392
:102228003B430B43611CC97F012905D1002A00D01B
:1022380078E0802252021343626A002A05D0E02126
:1022480049000A40A16A0A431343EA684A490A4016
:102258001343EB60230062683C33E16C1B78970FF3
:10226800BF079C463943012B08D1236C666C334366
:102278000B43A16C0B4361463B4319432B693F4F0A
:102288003B400B4380212B6153005B08C9058B42FF
:102298000CD080231B069A4208D03949394F0B6865
:1022A8003B40F027BF033A4013430B6007217027D8
:1022B8006B69626B8B4313436B616969A36BB943A9
:1022C8001B010B436B61002834D11023A96A5B42C0
:1022D8000B43AB6207216B690B409A4239D100234B
:1022E800E365A26D03339A43023B1343A365019848
:1022F80005B0F0BDAA6824490A401343AB60234BDC
:1023080023491868FDF70AFF013040000390039B3A
:10231800002B00D146E7039B013B0393F7E780219D
:10232800890377E72022A76D3A43A265E26D11433E
:10233800E16581E780239B039842CBD11C21AB6ADE
:10234800E369013B9B000B402C3999400B00216E3F
:10235800BEE71223A26D9A43023B1343A3650123F0
:10236800E26D1343E36501230193C0E7A36D1A43AC
:10237800A265F8E7FDFEFFFF0102DEFF02FCFF1F7A
:1023880008270140FFFFC3FFE8FFFF6F00000020A0
:10239800400D03007047704710B5806AFFF7FBFFD8
:1023A80010BD70474023806A10B5826D1343836562
:1023B8000423C26D1343C365FFF7F3FF10BD00008C
:1023C800502370B5846AA26D1A422DD1A26DB13323
:1023D800FF331343A365C02325681B01EA681A422B
:1023E80015D1A37E002B12D12B681B070FD528000F
:1023F800FFF7BCFE00280ED10C226B6893436B607C
:10240800A26D0F4B1A400433FF331343A36520001A
:10241800FFF7C0FF70BD2023A26D1343A3650123FE
:10242800E26D1343E365F2E7A36DDB0603D52000F5
:10243800FFF7B7FFEEE7236D5B6B9847EAE7C04607
:10244800FEFEFFFF0023F0B585B003930300009163
:1024580054331A7804000220012A4CD0012227693B
:102468001A7025682800FFF781FE002800D0E9E0EF
:10247800009B04225B6880219C4697436246009B30
:1024880009061B68022A00D1B0E05A03520B8F429A
:1024980033D1A96A0A43AA62009A68699268190244
:1024A8006B4E0A403240884302436A61002B1EDAB1
:1024B800E021684A6848156849042940834200D0E9
:1024C8007EE080200004054211D11368634D2B4043
:1024D8000B431843624B106018686249FDF71EFEF3
:1024E800431C0C2058430390039B002B64D100200D
:1024F80000235434237005B0F0BD1F2167460F40F8
:102508001039B940CE430196266E8E433100002A19
:1025180012D1980E1F321040B84062460843920804
:10252800E169013220668A42B6D8A96A01989A0000
:10253800120FBA400140ADE701221342ECD19218C4
:1025480001201342E8D1100002321342E4D10130D5
:102558001A07E1D40130DA06DED401309A06DBD45A
:1025680001305A06D8D401301A06D5D40130DA051C
:10257800D2D401309A05CFD401305A05CCD40130D9
:102588001A05C9D40130DA04C6D401309A04C3D478
:1025980001305A04C0D401301A04BDD40130DA0322
:1025A800BAD401309A03B7D480221800D20210405E
:1025B8001342B1D01220AFE7039B013B039393E78B
:1025C800294883420BD180204004054200D08EE781
:1025D8001368224D2B400B431843106087E72348AC
:1025E800834200D083E78020C003EEE78F4204D106
:1025F800AA6A5903490B8A43AA62002B00DB76E7D3
:10260800144A15481168834208D1A02310685B0456
:102618000B40124901400B43136068E7124883429C
:1026280003D1C02310681B04F2E71048834200D08E
:102638005DE7C0204004136801400848034019437F
:10264800116054E72023A26D01201343A3654FE7CF
:1026580000FFFF0708270140001000B0FFFF3FFE02
:1026680000000020400D0300004000B8002000B426
:1026780070B5056804002800FFF778FD002801D12F
:10268800002070BDAB689B0705D4AA680F4B1A40A1
:1026980010231343AB60FFF763FD0426050023688E
:1026A8009B683342ECD0FFF75BFD401B0228F6D94C
:1026B80023689B683342F2D010230120A26D134394
:1026C800A365E36D0343E365DBE7C046E8FFFF7FEF
:1026D8000023F7B502680193916801330400194299
:1026E80001D00020FEBD90682249084208D010227F
:1026F800A16D0A43A265E26D13430120E365F1E78A
:1027080091681D4F39400B4393601C4B1B681B029B
:1027180021D4637E012BE4D0FFF722FD01250600BA
:10272800226813682B42DCD193682B4203D193684B
:102738003B402B439360FFF713FD801B0228EFD922
:1027480023681B682B42EBD11023A26D1343A365AA
:10275800E36D2B43D1E70A4B0A491868FDF7DEFC05
:1027680001300190019B002BD3D0019B013B0193C9
:10277800F8E7C04617000080E8FFFF7F0827014000
:1027880000000020400D0300F7B50568040028008C
:102798000E000192FFF7EAFC022300283FD1270030
:1027A80054373A78012A3AD0013B3B70EA681A421A
:1027B8000CD1AA681A4205D0AA681A4B1A400223FB
:1027C8001343AB600123EA681343EB602000FFF773
:1027D8007FFF031E23D1A16D134A114080225200AE
:1027E8000A43A265E065114A206D2168C262104A59
:1027F8000263104A42631C220A603B704A68103325
:1028080013434B603200019B403100F0C7F90300CD
:102818002068044A8168114004220A438260180033
:10282800FEBDC046E8FFFF7FFEF0FFFFC92300089A
:10283800A1230008AD2300080122036870B5040035
:1028480098689968114201D1002070BD02210842A0
:10285800FAD105209D680540012D1ED19A681348BC
:1028680002401143032299601A60FFF779FC0600C1
:1028780023689B682B42E7D0FFF772FC801B022875
:10288800F6D923689B682B42F2D01023A26D13431C
:10289800A365E36D2B43E36506E01023A16D0B43AD
:1028A800A365E36D1A43E2650120CEE7E8FFFF7FE9
:1028B80070B506005436337804000225012B26D063
:1028C80001233370FFF7D4FE051E1ED1206D831D32
:1028D800DB7F022B08D100F0A9F9002804D040239F
:1028E8000500A26D1343A3651021226820005368D8
:1028F8008B435360002D0CD1FFF79EFF051E0BD0B4
:1029080001212268D3688B43D360002333702800E9
:1029180070BDFFF791FFF3E7A26D034B1A40043334
:10292800FF331343A365EBE7FEFEFFFF10B5FF245B
:1029380003220B0021000240D20091409B0123405A
:10294800C943934000280ADBC0240B4A8008800052
:102958008018A40002590A401343035110BD0F22E6
:1029680010400838054A800880008018C269114064
:102978001943C161F2E7C04600E100E000ED00E064
:10298800002805DB1F2318401E3B8340014A1360C3
:102998007047C04600E100E0002809DB1F2318400B
:1029A8001E3B8340034AD367BFF34F8FBFF36F8F3C
:1029B8007047C04604E100E08022431E5204012013
:1029C80093420DD2C021074A07485360036A09069B
:1029D8001B021B0A0B43036200200723906013604D
:1029E8007047C04610E000E000ED00E0F0B5846CF0
:1029F800C56C6560046D002C02D0446D856D656002
:102A08001C24056C084E25401B3CAC4077683C43B1
:102A18007460046863608368102B02D1A260E1606F
:102A2800F0BDA160E260FBE70000024010B50400C1
:102A3800036C094A9B089B189B0043640068142197
:102A4800C0B20838FDF76AFB044BA3641F23184083
:102A58001E3B8340E36410BD0082001080080240E2
:102A6800F8B504000120002C46D02568254B142118
:102A7800E818FDF753FB02238000A61D2064F377B6
:102A88002B68214AA76813402B60E36821693B4300
:102A98000B4361692A680B43A16920000B43E16974
:102AA8000B43216A0B4313432B60FFF7BFFF8023BF
:102AB800DB019F4201D1002363603F236268616CA0
:102AC80013400B60E06CA16C013A4860032A14D8EB
:102AD8000E4A0F4899180122013B9A40A26513003B
:102AE80000228900216560650A6043600020012397
:102AF800E0630534F377E077F8BD00232365636569
:102B0800A365F3E7F8FFFDBF0F80FFFF3F820010CA
:102B180040090240F8B5012504002800002C34D0F3
:102B2800276814213B680026AB433B60174BF81815
:102B3800FDF7F4FA1C238000206418402B00834022
:102B4800134A3E60516820000B435360FFF76EFF45
:102B5800636CE26C1E60A36C5A6063685A1E032A99
:102B680006D895400B495B189B001E600A4B5D60B8
:102B78000020A31D20656065A065E0622063606396
:102B8800A063E0630534D877E077F8BDF8FFFDBFB0
:102B9800000002403F82001040090240F7B5451D81
:102BA8000193EE7F04000220012E33D00138E8772C
:102BB800A71DFE7FB4466346F6B200960026834200
:102BC80030D10130F8772568E6632868009B984380
:102BD8002860019B2000FFF709FF236BB3421AD03E
:102BE8000E232A6813432B60636C1A68D20304D53A
:102BF8008022196852000A431A60236D002B04D002
:102C08008022196852000A431A60012300202A68AA
:102C180013432B60FEBD04222B6893432B602A6864
:102C28000A23DFE78023E363EE77F3E7F0B50028B4
:102C380008D0841DE37F411D022B05D00423C36304
:102C48000023CB770120F0BD0E250268466C13687F
:102C5800AB4313603368104D2B4033600123166873
:102C68009E431660026C1B331A401B3B93400B4E6D
:102C780077683B437360C26C836C5A60036D002BAA
:102C880005D01A682A401A60436D826D5A60012384
:102C98000020E377C877D6E7FFFEFFFF0000024079
:102CA800F8B5811DCB7F022B03D00423C363012019
:102CB800F8BD0E2402681C271368456CA3431360F3
:102CC800012314689C4314602A68104C22402A602F
:102CD800026C0F4D3A4093406E6833436B60C26C90
:102CE800836C5A60036D002B05D01A6822401A6065
:102CF800436D826D5A6001230022CB77431DDA773A
:102D0800836B934200D098470020D1E7FFFEFFFF76
:102D180000000240F8B51C240427016C264A214013
:102D28003C008C40166803681D6826420FD03D425F
:102D38000DD01968890602D41968B9431960536817
:102D48001C43036B5460002B1BD0984719E00227E3
:102D58003C008C40264215D03D4213D019688906A4
:102D680006D40A251968A94319600121831DD9775A
:102D780053681C4354600022431DDA77C36A9342A8
:102D8800E3D1F8BD082427008F403E42F9D0254200
:102D9800F7D00E251C68AC431C6001231D008D4034
:102DA8002900546821435160821DC363D3770022F0
:102DB800431DDA77436BE2E7000002400630C07F2C
:102DC800C0B27047C06B70470020054B5A698242F9
:102DD80005DA044A9A60044A9A605869C00F704735
:102DE8000020024023016745AB89EFCDF8B5040008
:102DF800FFF7B6F9802706007F02144D2B693B4286
:102E080016D12A69124B11001248194028611A423A
:102E180017D18027FF022B69180038403B420FD09A
:102E2800631CF8D0FFF79CF9801BA042F3D306E09F
:102E3800631CE3D0FFF794F9801BA042DDD3032085
:102E4800F8BD054B01205960FAE7C0460020024052
:102E5800FA830000FB83000008030020F7B5174E33
:102E68000193337804000D0002200092012B1ED03C
:102E78000123FA203370002380007360FFF7B6FF48
:102E8800002812D10E4F012C12D17B6923437B619C
:102E9800009B2B60BFF36F8F019B6B60FA20800053
:102EA800FFF7A4FF7B69A3437B6100233370FEBD5A
:102EB8002800009903F028FCF0E7C046080300202A
:102EC80000200240FA2010B58000FFF78FFF802213
:102ED800044B120659690A435A615869C043C00F26
:102EE80010BDC04600200240044A05485369C90085
:102EF80003401943034B0B435361704700200240C2
:102F080007E0FFFF02000100F7B5214F05003B78FD
:102F180002240191012B1AD00123FA203B700023CF
:102F280080007B60FFF762FF041E0ED104236B60F4
:102F38002B68042B0DD1FA20164A174B51698000D3
:102F48000B435361FFF752FF040000233B7020003E
:102F5800FEBD0123019A5B421360AE68AB68EA6864
:102F68009B18B3420CD968683100FFF7BDFFFA20FF
:102F78008000FFF73BFF002808D00400019B1E607B
:102F88000221044A53698B435361DEE70136E5E7C2
:102F98000803002000200240040001000023F0B5CF
:102FA80085B00A681400DC4001D105B0F0BD0125E8
:102FB80014009D402C4000942A4200D191E04A68B8
:102FC8005F0094460322644622400324BC40E44345
:102FD8000194541E012C2ED88668019C2640CC688A
:102FE800BC403443846044680126AC4325006446F1
:102FF800240934409C402C434460C568019C25400A
:103008008C68BC402C43C460022A16D107250F26C1
:103018001D40AD00AE40DC08A40004190294246AE7
:1030280003962600039CA64334000E69AE4026434F
:10303800029C266201E0032ADFD1BA400468019DA0
:1030480025402A43C02402606246A402224248D096
:10305800254A03259C08A400A4180F221D40ED0052
:10306800AA40A027266EFF0596430022B8420CD03E
:103078001E4F0132B84208D01D4F0132B84204D069
:103088001C4F0332B84200D1023AAA406746324385
:103098002266154C009A2668009DD2433543FF02EC
:1030A80001D435001540674625606668009D3543A4
:1030B800BF0201D435001540674665600E4C009D7F
:1030C800E66F3543BF0301D4350015406746E56711
:1030D8000A4C009EE56F2E43FF0301D415402E00D5
:1030E800E66701335DE7C04600180240000400505F
:1030F80000080050000C0050081802400418024054
:10310800F0B500230F0085B03A00DA4001D105B0D0
:10311800F0BD01229A40140001923C40174253D05E
:103128002A4903259A08920052180F211D40ED00E4
:10313800A940166E02910E400396A0260021F605BE
:10314800B0420FD022498C46012160450AD021495E
:103158008C460221604505D01F498C4603216045F5
:1031680000D00231A940039DA94212D11B4E174934
:10317800F56FA543F5671A4EF56FA543F5674D68DA
:10318800A5434D600D68A5430D60116E029CA143D7
:103198001166032459008C4007210F261940890025
:1031A8008E400268019922430260DA089200821870
:1031B800156AB54315628268A243826042688A43F1
:1031C8004260C268A243C26001339DE70018024012
:1031D8000004005000080050000C00500418024081
:1031E8000818024000690840431E9841C0B2704761
:1031F800002A01D0816170478162FCE742691300AF
:103208000B401B0491430B438361704770B5084D15
:103218000400EB68184202D0E86002F0CFF92B698D
:10322800234203D020002C6102F0BCFA70BDC046D6
:103238000018024070B504000120002C16D0236845
:10324800124A07261A60124A1A6062685A60A2680F
:103258009A60FEF785FF05002368DA68324206D1D6
:103268001969E26891420DD01A61002070BDFEF71D
:1032780077FF401B3128EFD92368DB683342EBD056
:103288000320F3E7034A1A60EFE7C046CCCC0000FE
:1032980055550000AAAA00000368024A00201A60D7
:1032A8007047C046AAAA000010B5114C11492368FE
:1032B80002000B4003432360802300209B009A42B6
:1032C8000ED10D4B0D49186806235843FCF726FF0D
:1032D8008022431CD200616908001040114200D1CD
:1032E80010BD002B01D0013BF5E70320F8E7C046ED
:1032F80000700040FFF9FFFF0000002040420F006F
:10330800F0B5040085B0002802D1012005B0F0BD59
:103318000368DB0710D423689B075CD423681B076A
:1033280000D5C1E023685B0700D5F2E0E369002B14
:1033380000D079E10020E9E73822AF4DAB681340AF
:10334800EA68102B09D1D3439B0708D12B689B034C
:10335800E1D56368002BDED1D7E7082BF6D08022B1
:1033680063685202934211D12A6813432B60FEF717
:10337800F7FE80270600BF022B683B42CBD1FEF741
:10338800EFFE801B6428F7D90320BFE7A021C902FC
:103398008B4208D180232968DB020B432B602B6802
:1033A8001A432A60E3E72A6894490A402A602A688F
:1033B80093490A402A60002BD9D1FEF7D1FE802715
:1033C8000600BF022B683B42A5D0FEF7C9FE801B52
:1033D8006428F7D9D8E73822874DAB681340EA68E4
:1033E800102B28D103210A40022A26D12A68520527
:1033F80003D5E268002A00D187E7696862698148D5
:10340800120201400A436A60002B0CD12B687E4AE5
:103418007E491340226913432B602B687C4A9B0426
:103428005B0FDA400A607B4B1868FEF751FE0028F4
:1034380000D173E769E7002BD8D0E368002B20D0D0
:103448002B68714A802713402269FF0013432B60C1
:1034580080232A685B0013432B60FEF781FE060079
:103468002B683B4207D06A68636966491B020A40B9
:1034780013436B6052E7FEF773FE801B0228EFD9F7
:1034880082E72B68644A802713402B60FEF768FEAA
:103498000600FF002B683B4200D13FE7FEF760FEC5
:1034A800801B0228F6D96FE73822534DAB681340CA
:1034B800182B08D12B6E9B0700D433E7A369002B88
:1034C80000D02FE721E7A2690123002A10D02A6E35
:1034D800022713432B66FEF743FE06002B6E3B4282
:1034E80000D01FE7FEF73CFE801B0228F6D94BE709
:1034F8002A6E02279A432A66FEF732FE06002B6ED2
:103508003B4200D10EE7FEF72BFE801B0228F6D9BE
:103518003AE73822384DAB681340202B08D1EB6DC1
:103528009B0700D402E7A368002B00D0FEE6ECE678
:1035380080220021EB6B52050091134208D1EB6BFE
:103548001343EB63EB6B13400393039B012300933B
:103558008027324E7F0033683B4215D0A368012B89
:1035680022D1EA6D1343EB65FEF7FAFD0227060048
:10357800EB6D3B4238D0009B012B00D0D6E6EB6BBD
:10358800274A1340EB63D1E633683B433360FEF7C9
:10359800E7FD019033683B42E0D1FEF7E1FD019B76
:1035A800C01A0228F6D9EFE6EA6D052B05D1013BD2
:1035B8001343EB65EA6D0123D4E701218A43EA65E9
:1035C800EA6D03318A43EA65002BCDD1FEF7C8FDC9
:1035D80002270600EB6D3B42CDD0FEF7C1FD114B33
:1035E800801B9842F6D9CFE6FEF7BAFD0D4B801B3B
:1035F8009842BDD9C8E6C04600100240FFFFFEFF52
:10360800FFFFFBFFFF80FFFFFFC7FFFF0000002059
:103618000024F40008000020FFFEFFFF00700040B7
:10362800FFFFFFEF8813000038213F4DAA680A40CA
:10363800102A51D03D4A022B38D12B6880271340DD
:103648002B60FEF78DFD0600BF042B683B4227D197
:10365800616A236AEA680B43354980260A401343A6
:10366800E26AB6041343226B1343A26A120213439D
:10367800EB6080232A685B0413432B608023EA688D
:103688005B051343EB60FEF76BFD04002B683342C8
:1036980000D04FE6FEF764FD001B0228F6D973E65A
:1036A800FEF75EFD801B0228CFD96DE62B688026C9
:1036B80013402B60FEF754FD0400B6042B68334218
:1036C80004D1EB681B4A1340EB6033E6FEF748FD74
:1036D800001B0228F2D957E6012B00D115E6032278
:1036E800E868216A02408A4200D00EE67022616AC8
:1036F80002408A4200D008E6FE21A26AC9010140C0
:103708001202914200D000E6F822E16A92030240D8
:103718008A4200D0F9E5236B400F4007C01A431EC8
:103728009841C0B2F2E5C04600100240FFFFFFFE1C
:103738008C80C11FFCFFFEEF382370B51D4CA268BA
:103748001A4205D123681C489B045B0FD84070BD02
:10375800A2681A40082A27D0A2681A40102A17D14E
:10376800E368E168DB43E5684906490F6F322D0AD3
:10377800013115409B0709D11048FCF7CFFCE168DF
:103788006843490F0131FCF7C9FCE0E70A48F4E750
:10379800A2681A40202A09D0A26800201340182BDA
:1037A800D5D1FA20C001D2E70448D0E78020000232
:1037B800CDE7C046001002400024F40000127A0051
:1037C800F7B504000D00002801D10120FEBD072730
:1037D8004A4E33683B408B422AD3226893073BD436
:1037E800D20748D4072733683B40AB420AD933682D
:1037F800BB432B433360FEF7B3FC019033683B4077
:10380800AB426BD123683E4D5B076FD4FFF794FF43
:10381800AB683C491B051B0F9B005B581F210B40E5
:10382800D840394A394B10601868FEF751FCCDE78B
:103838003368BB430B433360FEF792FC0190336857
:103848003B40AB42C9D0FEF78BFC019BC01A304B02
:103858009842F4D90320B9E72949530704D5E0234E
:103868008868DB0103438B608B682A480340A068A3
:1038780003438B60B4E76268214F012A19D13B6882
:103888009B03A2D50721BB688B431343BB60FEF79C
:1038980067FC01903823BA681A406368DB009A42D3
:1038A800A0D0FEF75DFC019BC01A194B9842F1D9D4
:1038B800D0E7022A03D13B689B01E3D485E7002ABD
:1038C80003D13B685B05DDD47FE70223032A03D1DC
:1038D800396E1942D6D178E7F96DFAE7FEF740FC60
:1038E800019BC01A0A4B984288D9B3E7AB680A4AC9
:1038F8001340E2681343AB6088E7C04600200240EB
:103908000010024080670008000000200800002026
:1039180088130000FFF0FFFFFF8FFFFF064B0749EA
:103928009B68074A5B045B0F9B005B581F2110686C
:103938000B40D8407047C04600100240606700083E
:1039480000000020F0B50368050085B000209B0347
:1039580051D58022484C5205E36B0090134208D1A0
:10396800E36B1343E363E36B13400393039B01236C
:1039780000938027414E7F0033683B433360FEF756
:10398800EFFB019033683B4227D0E16DC02208006D
:1039980092006B691040114217D098420CD0E36D29
:1039A800374AE16D1340802252020A43E265E26D14
:1039B80034490A40E265E365DB0706D5FEF7D0FB2C
:1039C80002270600E36D3B424ED0E36D2C4A0020EF
:1039D80013406A691343E36506E0FEF7C1FB019BE8
:1039E800C01A0228CED90320009B012B03D1E36B18
:1039F800254A1340E3632A68D30706D503241E49E2
:103A08004B6DA3436C6823434B65930606D51A494F
:103A18001E4C4B6D2340AC6823434B6553040FD5B4
:103A280015492C694B6D9B009B0823434B658023EC
:103A3800DB059C4204D18023CC685B022343CB6026
:103A480012050FD50C4A124C536DE96823400B43FD
:103A580053658023DB01994204D18023D1685B023E
:103A68000B43D36005B0F0BDFEF77AFB094B801B12
:103A78009842A7D9B7E7C04600100240007000403E
:103A8800FFFCFFFFFFFFFEFFFFFFFFEFFFCFFFFF82
:103A9800FF3FFFFF8813000070B50124036A026A24
:103AA800A24302624468164A856915400A681543AC
:103AB800022293438A681343124A904205D0124E59
:103AC800B04202D0114EB04213D10826B343CE689B
:103AD80033430426B343904205D00B4A904202D0A8
:103AE8000A4A904205D10A4A8E6922404C693443F9
:103AF80014434A68446085614263036270BDC046EE
:103B08008CFFFEFF002C01400044014000480140AA
:103B1800FFFCFFFF70B5174A056A036A134003628A
:103B28004268154BC4691C400B681C43134B1D406D
:103B38008B681B022B43124DA8420ED1114D1D401C
:103B4800CB681B022B43104D2B40104D4E6915407E
:103B58008A69324312012A4305E00D4DA842F4D088
:103B68000C4DA842F1D042604A68C461C263036246
:103B780070BDC046FFFEFFFF8CFFFEFFFFFDFFFF8D
:103B8800002C0140FFF7FFFFFFFBFFFFFFCFFFFF08
:103B9800004401400048014030B5124A046A036AF3
:103BA800114D134003624368C2692A400D682D0213
:103BB80015430E4A14408A68120322430C4CA04253
:103BC80005D00C4CA04202D00B4CA04204D10B4CA7
:103BD8001C404B699B01234343604B68C5610364E8
:103BE800026230BDFFEFFFFFFF8CFFFEFFDFFFFF2C
:103BF800002C01400044014000480140FFBFFFFF86
:103C080070B5066A104C036A104A23400362436881
:103C1800456D15400A6815430D4A16408A68120416
:103C280032430C4EB04205D00B4EB04202D00B4E80
:103C3800B04203D11C404B691B02234343604B68CD
:103C480045658365026270BDFFFFFEFF8FFFFEFFC3
:103C5800FFFFFDFF002C01400044014000480140E7
:103C680030B5124A046A036A114D1340036243686F
:103C7800426D2A400D682D0215430E4A14408A6889
:103C8800120522430C4CA04205D00C4CA04202D095
:103C98000B4CA04204D10B4C1C404B699B022343A4
:103CA80043604B684565C365026230BDFFFFEFFFA7
:103CB800FF8FFFFEFFFFDFFF002C014000440140A3
:103CC80000480140FFFFFBFF01000300012010B581
:103CD8003D310C78E2B2844218D1001808701B6894
:103CE800D9681143D9600B498B4202D00A498B42EB
:103CF8000DD19A6809490A40062A06D007398A422E
:103D080003D0012219680A431A60002010BD1968FF
:103D1800F9E7C046002C01400004004007000100FC
:103D2800704700001C4A10B50368904202D01B4C33
:103D3800A04208D17024A3434C68234390420BD07F
:103D4800164CA04208D0164CA04205D0154CA042F3
:103D580002D0154CA04203D1144C1C40CB6823431D
:103D68008024A3434C69234303608B68C3620B68B8
:103D78008362904205D00B4B984202D00A4B98427E
:103D880001D10B690363012242610369134202D026
:103D980003699343036110BD002C014000040040F7
:103DA800002000400044014000480140FFFCFFFFA4
:103DB80070B504000120002C23D025003D352B7858
:103DC800DAB2002B05D123003C3320001A70FEF72D
:103DD80003F802232B702068211DFFF7A3FF2200A0
:103DE800012300204832137047340A3A1370537085
:103DF8009370D370137153719371D37113722370CD
:103E08002B7070BD70B504000120002C23D0250054
:103E18003D352B78DAB2002B05D123003C33200046
:103E28001A70FFF77DFF02232B702068211DFFF712
:103E380079FF2200012300204832137047340A3AE0
:103E4800137053709370D370137153719371D3714E
:103E5800137223702B7070BD102270B5056A036A47
:103E6800164C934303624268836923400C6824021A
:103E78001C4320239D438B681B012B43104DA842F4
:103E88000FD18025AB431E00CB68403D1B01334357
:103E9800AB430C4D4E6915408A69324392002A4360
:103EA80005E0094DA842F4D0084DA842F1D042607F
:103EB8004A6884618263036270BDC046FF8CFFFE5E
:103EC800002C0140FFF3FFFF00440140004801407F
:103ED800F8B507003C3715003A7803000C000220BB
:103EE800012A0CD0013838700C2D51D008D8042D77
:103EF8002DD0082D3CD0002D17D000233B70F8BDE5
:103F0800102D58D0142DF8D11D682800FFF7A8FEF1
:103F180080236A6D1B0113436B656B6D2E4A13403A
:103F28006B6523696A6D1B0253E01D682800FFF763
:103F3800B3FD0823AA6913430422AB61AB69934319
:103F4800AB61AB6922691343AB610020D5E71D68FB
:103F58002800FFF781FF8023AA691B011343AB6187
:103F6800AB691D4A1340AB612369AA691B02EAE7E2
:103F78001E683000FFF7CEFD0422F3691D43F5618A
:103F8800F3699343F361F36922691343F361DCE74F
:103F98001D682800FFF700FE8023EA691B01134310
:103FA800EB61EB690C4A1340EB612369EA691B0278
:103FB8001343EB61C9E71D682800FFF721FE0823BA
:103FC8006A6D134304226B656B6D93436B656B6D70
:103FD800226913436B65B8E7FFFBFFFF1F2310B58A
:103FE800012419408C408A40036AA3430362036A90
:103FF8001A43026210BD000010B508291CD006D86B
:1040080000290BD0042914D00300433308E00C29FD
:1040180015D01029F8D10300423301E003003E33E4
:104028001B78013B5A1E9341DBB2002B0AD00120BA
:1040380042E003003F33F3E703004033F0E70300B7
:104048004133EDE7022308293ED009D800290ED0D4
:10405800042932D00200433213700429E7D12FE03B
:104068000C2939D01029F5D142300370DFE702005E
:104078003E3213700468E2681343E3600468012267
:104088002000FFF7ABFF1C4A94422DD01B4B9C42EB
:104098002AD01B4B9C4227D01A4B9C4207D1A368BD
:1040A800194A1340062B06D0073A934203D001233E
:1040B800226813432360002010BD02003F321370B2
:1040C80002680423D4680DE00200403213700268CD
:1040D800D3680B43D360D1E7020041321370102339
:1040E8000268D4682343F5E78023616C1B020B4305
:1040F80063649442D3D0CFE7002C014000440140D0
:1041080000480140000400400700010010B5FFF717
:1041180073FF10BD30B5EFF31084012282F31088CD
:10412800C02501680B68AB430B6084F31088EFF37C
:10413800108182F310880268044C936823409360CE
:1041480081F3108820238830036030BDFFFF7FFF94
:1041580030B5EFF31084012282F310880168134D03
:104168000B682B400B6084F31088EFF3108182F307
:10417800108802680E4C93682340936081F310887E
:10418800C36E012B0AD1EFF3108183F3108810243A
:1041980002681368A343136081F310880300202288
:1041A8008C331A600023C366436730BDDFFEFFFF10
:1041B800FEFFFFEF70B505000120002D19D02E007D
:1041C80024230024883633602B681A6882431A60D7
:1041D80028001C605C609C60FDF72EFF2B0020000F
:1041E80090331C60043B34601C60EC662C6784359B
:1041F8002C7070BDF7B50500883513002A680400D7
:104208000220202A04D1002901D0002B01D101204D
:10421800FEBD8022A0685201904204D12269002A82
:1042280001D1CA07F3D422002600543221650027A1
:1042380013805380212290363760E06F2A6022680D
:104248000192B84211D0114A8763C262104A0263D0
:10425800104A4263019A2832FEF7A0FCB84204D003
:1042680010233360DB182B60D1E7402223681A62E1
:10427800EFF31081012383F3108822687F3390685D
:104288000343936081F310880020C1E74943000885
:104298009B430008AB4300080300020080218C32D6
:1042A800883370B51B6815680268040092680A4272
:1042B80020D0212B1ED1EFF31080203B83F31088F0
:1042C800226893688B43936080F31088E06F00281E
:1042D8000DD0FEF7ABFC002809D0E06FFEF772FDA9
:1042E800202804D110239034032023600AE0200002
:1042F800FFF710FF402123689B680B4201D0222D55
:1043080001D0002070BDEFF31080012383F31088E3
:10431800250004CD93688B43936080F31088E86F81
:10432800002808D0FEF782FC002804D0E86FFEF7CA
:1043380049FD2028D6D02000FFF70AFFE1E77047A3
:1043480003001B6870B51A6820231100806A1940A1
:104358001A421AD1030056331980EFF31084012250
:1043680082F31088802501688B68AB438B6084F3E7
:104378001088EFF3108182F31088402302681068D8
:104388000343136081F3108870BDFFF7D8FFFBE784
:10439800704710B5806AFFF7FBFF10BD7047704784
:1043A800704770B5846A230088331A685D6823688B
:1043B8009B681B0608D5212A06D123000022563304
:1043C80020001A80FFF7A6FE23689B685B0608D5C5
:1043D800222D06D1230000225E3320001A80FFF729
:1043E800B7FE220010239032116820000B4313609F
:1043F800FFF7D6FF70BD806A0023020010B55E3259
:104408001380083A1380FFF7CBFF10BD70470000F8
:10441800F7B50168C14DCB6904000A6888682B426A
:1044280010D120252B4200D19BE08026760515402F
:104438000640354300D194E0636F2000002B00D084
:1044480085E085E0B64D05400095B64D009E1540C7
:10445800354300D185E0250001269035334205D04B
:10446800D70503D50E622F683E432E6002263342DD
:104478000CD0C7070AD527000E6290373E6801970F
:10448800B446042667463E43019F3E6004263342F5
:104498000CD0C7070AD527000E6290373E680197EF
:1044A800B446022667463E43019F3E600826B4464E
:1044B800334209D02027009E1740374304D0664670
:1044C8000E622F683E432E6080263601334206D0A6
:1044D800570104D50E6220212E68314329602968CE
:1044E800002935D020210B420AD080235B051140DA
:1044F8000340194304D0636F002B01D02000984774
:1045080022682B684027966828223E4013402000E6
:104518001E4322D0FFF71CFE23689B683B4218D03D
:10452800EFF31081012383F31088250004CD9368ED
:10453800BB43936081F31088E86F002809D07A4B59
:104548008363FEF7ADFB002802D0E86F836B9847C2
:10455800F7BD2000FFF724FFFAE7FFF721FF2E60E1
:10456800F6E7E56E012D00D09FE01026334200D11A
:104578009BE0324200D198E00E62896840230A002D
:104588001A40194257D0211DCA6F1068426892B26A
:10459800002ADDD027005C373F889742D8D927000A
:1045A8005E373A80026820208446104000906046BA
:1045B800024232D1EFF3108785F3108820685B4EF2
:1045C80002683240026087F31088EFF3108785F3A2
:1045D800108820688268AA43826087F31088EFF306
:1045E800108785F31088206882689A43826087F371
:1045F8001088230062468C331A60009BE366EFF351
:10460800108085F3108822680F351368AB43136058
:1046180080F31088C86FFEF709FB02232200236786
:1046280023005C325E331B881188C91A89B22000C6
:10463800FFF7ECFE8CE7230020005C335E3019881E
:10464800038800889BB2002800D181E7C91A89B283
:10465800002900D17CE7EFF3108785F310882068E4
:10466800334E03683340036087F31088EFF31087F5
:1046780085F3108820682F4E83683340836087F362
:104688001088230020208C331860E2666267EFF3FD
:10469800108085F31088102522681368AB431360D7
:1046A80080F3108802232367C1E780256D032B421E
:1046B80006D0460204D520000D6200F053FB47E700
:1046C80080210B4207D080252D041140284001434A
:1046D80001D0A36FB1E640210B4216D00A4214D094
:1046E800EFF31080012383F31088226813688B434B
:1046F800136080F310882300202288331A60002377
:104708002000A367FFF71BFE22E7190214D551000A
:1047180012D5200000F028FB1AE7C0460F08000059
:104728000100001020010004FF430008FFFEFFFF06
:10473800DFFEFFFFFEFFFFEFDB0100D408E7002AE2
:1047480000DB05E7200000F00EFB01E70123806A8B
:1047580010B50367C36E012B06D103005C331988BB
:104768004908FFF753FE10BDFFF719FEFBE70000ED
:1047780003001B6820221B6870B51900806A11406D
:10478800134234D103005E331980EFF310850123FF
:1047980083F3108804681D4E21683140216085F339
:1047A8001088EFF3108583F310880468A168994393
:1047B800A16085F31088EFF3108483F310884025F7
:1047C80001688B68AB438B6084F3108803008C33DB
:1047D8001A60C36E012B0AD1EFF3108183F310889E
:1047E800102402681368A343136081F31088002320
:1047F8000367C36E012B05D103005C331988FFF7EB
:1048080005FE70BDFFF7CAFDFBE7C046FFFEFFFFD0
:1048180070B504002569A168036829436569C26900
:1048280029431868494D11432840014319605968C4
:104838004748256A0140E06801435960A1699868C2
:104848002943444D284001430F209960D96A814388
:10485800606A0143D96240498B4215D103213F4B1D
:104868005B6D0B40013B022B60D83D49C85C80233F
:104878001B029A422FD1082856D8FBF745FC5B55F6
:104888000E550B5555550F0036495B18591E8B416F
:104898001801ECE7FEF750FF4EE0334A616A334BEC
:1048A80049001000C95AFBF739FC656840006B08DD
:1048B800C0182900FBF732FC02002D4B103A9A422F
:1048C80032D80F23020000079A4393B2400F2268A0
:1048D8000343D36032E0082826D8FBF715FC1A25D5
:1048E80005251F25252522001F48626A1F4B5200F7
:1048F800D15AFBF713FC65686B08C0182900FBF751
:104908000DFC02001A4B103A9A420DD82368D86061
:1049180014E0FFF703F8002810D0E6E7FEF70CFFD5
:10492800F9E780200002E0E7012008E080231B026D
:104938009A42EED1FEF7F2FF021EAFD100200D4BD6
:10494800A36600236367A36770BDC046F369FFCF02
:10495800FFCFFFFFFFF4FF110038014000100240B5
:10496800C067000800BCFFBF0024F400C46700084B
:10497800EFFF000001000100836A30B51A0706D571
:104988000168284C4A682240846B22434A60DA074F
:1049980006D50168244C4A682240C46A22434A600A
:1049A8009A0706D50168214C4A682240046B2243C5
:1049B8004A605A0706D501681D4C4A682240446B74
:1049C80022434A60DA0606D501681A4C8A682240F2
:1049D800C46B22438A609A0606D50168164C8A6819
:1049E8002240046C22438A605A0610D50168134D90
:1049F8004A68446C2A4022434A6080225203944207
:104A080005D14A680E4C2240846C22434A601B063A
:104A180006D502680B4953680B40C16C0B435360C1
:104A280030BDC046FF7FFFFFFFFFFDFFFFFFFEFF1A
:104A3800FFFFFBFFFFEFFFFFFFDFFFFFFFFFEFFFC2
:104A4800FFFF9FFFFFFFF7FFF7B504000D001700FA
:104A580000932268D3692B405B1B59424B41BB42F0
:104A680001D0002026E0089B0133F3D0FDF778FB46
:104A7800009BC01A089B98422DD8002B2BD0236886
:104A88001A685207E5D52A004021403A8A43E0D007
:104A9800DA69082611003140019132420BD020001A
:104AA8001E62FFF755FB230090331E600023012090
:104AB80084342370FEBD8022D96912011142C8D006
:104AC8001A622000FFF744FB2300202290331A606B
:104AD800019B843423700320ECE70000030073B5C6
:104AE8000026040090331E60FDF73AFB236805009A
:104AF8001B681B071FD58021284B320000938903B0
:104B080003002000FFF7A0FFB04214D0EFF310819C
:104B1800012383F31088802022681368834313607D
:104B280081F310882300202288331A600320002391
:104B38008434237076BD260023688C361B685B0797
:104B480023D58021154B0022009320002B00C90398
:104B5800FFF77AFF002818D0EFF31080012282F3C4
:104B6800108821680E4D0B682B400B6080F310886D
:104B7800EFF3108082F3108821688B6893438B6071
:104B880080F3108820233360D0E723002022002000
:104B980088331A603260E0662067C8E7FFFFFF01CC
:104BA800DFFEFFFF70B5041E01D1012070BD0500B6
:104BB80088352B68002B04D1020084321370FDF76E
:104BC800B9F92423012122682B6013688B431360F1
:104BD800A36A002B02D02000FFF7CEFE2000FFF7CB
:104BE80017FE0128E1D0236807495A6820000A40C7
:104BF8002A215A609A688A439A60012219680A43EE
:104C08001A60FFF76BFFD1E7FFB7FFFFF8B5130096
:104C18000200060005005C3281650F001380222126
:104C2800002290368C3532602960011D0400C86F5F
:104C3800904213D01D498263C1621D493A00016345
:104C48001C49416321682431FDF7A8FF002805D0DD
:104C5800102301203360DB182B60F8BD2369002B7B
:104C68000BD0EFF31081012383F310882268FF3300
:104C780010680343136081F31088EFF31080012359
:104C880083F3108821688A681A438A6080F3108841
:104C9800EFF3108183F3108822683F339068034351
:104CA800936081F310880020D7E7C0467947000851
:104CB80055470008AB43000803008C3070B5046802
:104CC8000220202C25D10138002922D0002A20D00A
:104CD80080209C684001844205D11869002802D1CF
:104CE8000130014215D10020D866186840680002DA
:104CF8000CD5EFF31085012080F3108880201C6804
:104D0800C00426683043206085F310881800FFF738
:104D18007DFF70BDF7B50700436E04006A37002BAE
:104D280004D10120388068342080F7BD03680B4E19
:104D38009A689B680A4D5B0FF05CE95CC0000192C1
:104D4800FBF776FA019B38801B015B0FF05CE95C8E
:104D5800C000FBF76DFA80B2E5E7C046E4670008DB
:104D6800DC670008704770477047000070B50400A2
:104D78008434227803000220012A11D01D00242245
:104D8800012688352A601A6811681068B0431060D7
:104D98000448014000205866202311602B602070D1
:104DA80070BDC046FFFFFFDFF8B5050084350B0076
:104DB80029780222012915D00600012104688836C5
:104DC80022323260276822688A432260A168C900BB
:104DD800C9081943A160FFF79DFF2023002227601F
:104DE80033602A701000F8BDF8B5050084350A0054
:104DF80029780223012915D0060001210468883684
:104E080022333360276823688B432360A168064BED
:104E180019401143A160FFF77DFF2023276033600D
:104E280000232B701800F8BDFFFFFFF1002302706C
:104E3800FA22437152000B1C914200D2131CC3800A
:104E48007047F7B51F00490008AB1E78CBB2141E97
:104E58000190009316D000F037FF009800F0F6FF9D
:104E680000F076FF451E200000F0F0FF00F070FF14
:104E78006B425D41013843425841EDB22D182C0078
:104E880000F044FF00F020FF00980130C0B200F0AD
:104E9800DDFF00F05DFF012801D10134E4B2013EDD
:104EA800F6B2122E01D8002C05D000F02FFF019B7E
:104EB80020001C71FEBD300000F0FAFF3870013789
:104EC800EDE7F7B50C001E0008AB1D78019207004E
:104ED80000F0FAFE6000C0B200F0B8FF00F038FF42
:104EE8000400019800F0B2FF00F032FF01280ED153
:104EF800013C63425C41013400F008FFE0B23871C4
:104F0800FEBD307800F0A2FF00F022FF0136012C30
:104F1800F2D0013DEDB2122DF3D90024ECE7F0B543
:104F2800030041180825FF2031268B4200D1F0BD2F
:104F38001A7850402A0047B24400E0B2002F01DA44
:104F48007440E0B2013AD2B2002AF4D10133ECE75E
:104F580037B5438804000A339BB243800A2B5ED9D5
:104F68004279002A0CD101234371323303810300B3
:104F78000232017808330092AA32FFF7A2FF37BD48
:104F8800962B4CD9012A4AD10223050043711C35BE
:104F980005330178002200932B00FFF752FF237995
:104FA800002B38D106212800FFF7B9FFE31CDB7F6F
:104FB8008342E4D16722237F9343182BDFD1A07F5C
:104FC800637F0002184340BAE57F80B200022818C8
:104FD8000009FBF733FD1549FBF72EFAD6218905A1
:104FE800FBF72AFA0F2320631D40631CDB7FA21CFA
:104FF8002D02D07F5B191B02C018FBF71FFD0C495F
:10500800FBF71AFAD6218905FBF716FA0949FBF7C7
:1050180051FB6063B3E7002323636363AFE7E28870
:105028009A42ACD2002363716380A8E70000C842AB
:10503800000048430000484210220A4B10B51B6884
:1050480019680A431A6050221A6201F019FAFA2103
:1050580038220548C900FFF7E9FE0122034B1A7000
:1050680010BDC04670020020240300202A00002042
:10507800F7B52E4C0121228813004800205A984287
:1050880043D8051C904200D9151CAAB20131FA294F
:10509800F3D1934204DD264908881B189B1A0B801C
:1050A800244D2B785A1C2A70032B3DD9224B204FB4
:1050B8001C88224B05211E88214B24B21B7836B24E
:1050C8005BB201930023F85EFBF7B2F803B21D4808
:1050D8001D495843FBF7ACF80A216043FBF7A8F8D1
:1050E800019B80195843194B194A00B2188011784E
:1050F80001290CD117481988028809B212B29142C5
:105108000FDD1B881BB203800BE00300BEE712789B
:10511800002A06D110481988028809B212B29142B1
:10512800EFDB00233B802B70F7BDC046AA030020AD
:105138007203002071030020A00300209E030020BA
:105148002C000020E40C0000FF0F0000A803002042
:10515800A0050020A6030020A4030020F0B5082520
:10516800012602000B4F0C4801390B4B89B29942BA
:1051780000D1F0BD137858402B000400400834409B
:1051880001D0784080B2013BDBB2002BF5D101326F
:10519800EAE7C04601A0FFFFFFFF000010B50024AA
:1051A8008CB02100142207A8069401F06AFA3B4B40
:1051B8000021595E4B1C9BB2012B00D82100022311
:1051C800374A0293DB181088039312880B33049331
:1051D8000E3B0593120A06AB5A70324A18701088B3
:1051E80012889870120ADA702F4A1088128818717B
:1051F80012B212125A712D4A10881288987112B27E
:105208001212DA712A4A10881288187212B212120F
:105218005A72284A108898721288D98112B21212CA
:10522800DA72254A12889A81244A1178012904D110
:1052380023490988D98100211170224A12881A82CB
:10524800FDF7C2FD01A902A8FDF75EFE002805D002
:10525800FDF738FE012420000CB010BD0120069A8D
:10526800079B1949FDF7FAFD002803D0FDF72AFE30
:105278000324F0E70120089A099B1449FDF7EEFD85
:105288000028F3D10A9A0B9B11490130FDF7E6FD7E
:10529800041EEBD1FDF716FEDDE7C0460E780008C8
:1052A8009E050020A2030020A00300209E030020EA
:1052B8009A03002028000020260000207403002004
:1052C80094030020240000200078000808780008D3
:1052D8001078000810B5012383F31088FFF75EFFEC
:1052E800002383F3108810BD10B50400A02001220C
:1052F8002021C005FDF77CFF220009490948FEF777
:1053080079FF0948FDF75AFD0128FAD1043001F068
:105318006BF9A02000222021C005FDF769FF10BD10
:10532800C105002070020020B8010020F0B58D48AA
:1053380085B0C57883782D021D436BBA9BB2029362
:10534800437902791B02134306215CBA0393FFF7E2
:1053580005FF030ADBB20093C3B20193824B834A71
:105368001B8883495380834BA4B21B785BB293801C
:1053780000200B5E80480027C75F002B00D091E01B
:1053880093807E4B794E1B78F3807D4B1B8833814D
:105398007C4B1B8873817C4B1B88B3817B4B1B88A0
:1053A800F3817B4B1B8833827A4B1A787A4B120233
:1053B8001B7813437382794B1B88B382784B1B8805
:1053C800F3826B4B1B883383674A13881BB2D91748
:1053D8005B184B4073499BB28B420CD910881188DB
:1053E80000B209B2CB17C918594089B2FAF720FFA1
:1053F800C82343433383029B5C491B194F830E2BFD
:1054080069DC584B01989A79824200D085E0DA79B4
:105418000098824200D09CE0634E1A7832705B7824
:1054280073706300B370029B5A00E3B25218029380
:105438003100002302980231834243D15B00DFB27E
:10544800F91C3000C9B2FFF789FE6300F318D87061
:10545800A31C000A5B000537F054F8B2FFF744FFBD
:10546800FD231B029D425AD13E4B01999A798A42EB
:1054780053D1DA7900998A424FD14B4D1A7864009A
:105488002A705B78AC706B70484B1B881A0A052130
:105498002800EA702B71FFF761FE6871000AA87195
:1054A800072038E0D8171B1843409BB2BB4200DBEB
:1054B80067E73F4B1B88062B00D862E700239380E1
:1054C8000B805EE70027D05F013307124F708870AA
:1054D800DBB20232AEE7FF231B029D42C0D180231C
:1054E800039A5B009A4218D11E4B01999A798A4215
:1054F80013D1DB79009A93420FD100242D4D2A4E07
:1055080003E02B5D33550134E4B22800FAF7F4FDCB
:105518008442F6D3C0B2FFF7E7FE05B0F0BDFC2326
:105528001B029D42F9D10F4B019A9B799342F4D10A
:105538000C4B0099DA798A42EFD11A781A4D640037
:105548002A705B78AC706B701B4B00229B5E1A1242
:105558009DE7FD231B029D42DFD0013BFF3B9D429F
:10556800E6D0DAE7A1050020A80300207603002092
:10557800960300202B000020240000202A00002091
:10558800A2030020A00300209E0300209C0300200B
:105598009A03002098030020990300202800002087
:1055A800260000201C0C0000C1050020100000206F
:1055B80092030020120000200E000020F7B504001E
:1055C800A0204021C005FDF70DFE604B802118701A
:1055D800A020C0050193FDF705FE802C38D10128D5
:1055E80031D1FCF7BDFD5A4E05003368C31A072BAD
:1055F8000FD8FA210420890000F0B8FF554F3B78F6
:10560800012B06D1FA210220490000F0AFFF002348
:105618003B70019B35601B78012B03D14E4A1378F0
:10562800013313704D4A13780133DBB21370092B21
:1056380009D9494B4A491878022807D90120087026
:10564800002111701970474BDC60F7BDFF20F6E7A9
:10565800082CF8D10320444900F088FFA02021003D
:10566800C005FDF7BFFD0128EDD1404B404A414E32
:10567800187013883188404F5B1A40499BB20B80E1
:1056880013883188388809B21BB200B25B1A3C4DC6
:105698003C49834241DD10883B8800B21BB29C46DE
:1056A8000023EF5EC01B604537DD00270B783648C6
:1056B8000133DBB20B700770022B05D93348077032
:1056C800FA2B01D903230B70338831492B801388B7
:1056D80000254D5F1BB2D9175B184B409BB22B4876
:1056E8002C49AB4230DA33881BB2DE179B19734062
:1056F8009BB29D4228DD0B8801339BB20B80022BA5
:1057080003D90023037003330B80234B1B881BB280
:1057180013800278214B1A7095E700271A480F70FA
:1057280003780133DBB20370012BCDD91749013758
:105738000F701A490978002901D1194F3980FA2BBD
:10574800C2D903230370BFE70023DDE770030020FD
:105758006C0300202A000020690300206803002051
:105768002C0000200018024088130000A00500202B
:10577800A6030020A4030020280000209C0300208A
:105788006603002065030020640300202B0000202E
:105798002600002062030020A80300200C0000203F
:1057A80094030020010010B508280CD1A020C005E2
:1057B800FDF718FD002801D1034B1870034B044A6C
:1057C8001B881BB2138010BDA0050020A803002071
:1057D800A403002070B5264C05002000FEF7EAFC63
:1057E800012D3ED0022D3FD0033D6B425D41214B40
:1057F8006842184096239B01C0181F4B0C22236057
:10580800002360602000A360E36023616261A361FC
:10581800E36123626362A362FFF7C4F9002801D041
:10582800FCF766FA00212000FFF7BEFA002801D035
:10583800FCF75EFA00212000FFF7D6FA002801D015
:10584800FCF756FA2000FFF791FA002801D0FCF780
:105858004FFA1022236819680A431A6050221A6204
:1058680070BD9620C001C8E7E1200002C5E7C04628
:1058780070020020809C010000380140F7B5B74C49
:105888000621677923793F021F43E378A2781B0238
:10589800134320000093FFF761FC0600B04B06227B
:1058A80021001800019300F019FF019AF3B2360A9B
:1058B800F6B29371D671F02200997FBABDB2120187
:1058C800914228D1A2799A4213D1E379B34210D1F7
:1058D800013DF62D11D8A34E35883780ADB2FFF7BC
:1058E800F9FC002806D16378002B02D00820FFF7C6
:1058F800FBFCF7BDEDB23580FBE7FF23019A0621DB
:10590800200013715371FFF729FC019B9871000A5D
:10591800D8712378E8E780220099D20091421BD100
:10592800A2799A42E5D1E379B342E2D1FA239B0006
:105938009D42DED88C4D2C882F80A4B2FFF7CAFC7C
:10594800002800D098E00830FFF7CEFC874A2B8863
:1059580012689BB25363CCE7A022009938B2D200F8
:10596800914229D1A2799A42C3D1E379B342C0D1F5
:105978007F4B804AEB189BB29342BAD87E4C7F4B40
:10598800268819880A2309B25843FAF751FC053DBD
:1059980000B236B220800F2D00D8278023881BB292
:1059A800042BA6DD23881BB2142BA2DCFFF792FC84
:1059B80000289BD026809CE7C0220099D200914203
:1059C80020D1A2799A4200D093E7E379B34200D07C
:1059D8008FE7674BED18674BADB29D4200D988E75A
:1059E800674D002840D10830FFF77EFC012383F380
:1059F8001088BFF34F8F634B634ADA60BFF34F8F52
:105A0800C046FDE780220099120191421AD1A2797D
:105A18009A4200D06DE7E379B34200D069E7032DDD
:105A280000D966E7594D2C882F8024B2FFF752FC25
:105A3800002821D10830FFF757FC288800B2FFF76B
:105A4800C9FE56E7A02200991201914216D1A27907
:105A58009A4200D04DE7E379B34200D049E74C4B76
:105A68009D4200D945E74B4D2C882F8024B2FFF783
:105A780031FC002800D139E72C803AE7B0220099A0
:105A88001201914216D1A2799A4200D031E7E37906
:105A9800B34200D02DE73E4B3F4C9D4200D928E74A
:105AA8000023E55E2780FFF715FC002800D11DE7DD
:105AB80025801EE7C0220099120191423AD1A279AD
:105AC8009A4200D015E7E379B34200D011E7DC230E
:105AD800DC35ADB25B009D4200D90AE72F4C0022AD
:105AE800A35E00930123002818D0244B1D88FBF7E0
:105AF80005FE02000B0000202949FAF7E1FF2DB24C
:105B0800060028000F00FBF7F9FD0B000200390022
:105B18003000FBF7EFFAFBF7B5FD03B20122238053
:105B2800204B1A70FFF7D6FB002800D1DEE6009B59
:105B38002380DEE6D02200991201914200D0D8E6F7
:105B4800A2799A4200D0D4E6E379B34200D0D0E6F5
:105B5800DC2D00D9CDE6144CA2E7C046A1050020F3
:105B6800C10500209E050020A20300206C01002032
:105B7800E40C0000C8190000A0030020A8030020BE
:105B88009E03002000ED00E00400FA059A030020BF
:105B9800DC050000280000202600002094030020D7
:105BA80000805B40740300202400002010B50E4BD9
:105BB8000E491A7809888A420ED10D4909780829B0
:105BC8000AD15B78032B04D0062B04D1FFF756FECD
:105BD80001E0FFF7ABFB10BD002AFCD1044A1278A4
:105BE800082AF8D15B78EFE7A10500209E05002080
:105BF80001060020F7B52D4B1B785AB2002B02D1B5
:105C08002B4B1A80F7BD2B4B01930027DF5F002F2A
:105C180031D1294D294E28882988348809B2CB17D3
:105C2800C91801345940A4B2348000B289B2FAF7D5
:105C3800FFFA6E2340B25843214A1D4B188013883F
:105C4800E31A042BDEDD2B881E491BB29C46002379
:105C5800C85E63461B1AD8171B184340272B05DC60
:105C68001D2C03D92B880198378003803388138033
:105C78002B880B80C6E7012FC4D100220C4B0E4D98
:105C8800104C1A802B880020215E1BB25B1AD91792
:105C98005B184B40962149008B4203DD019B1A801B
:105CA800FFF718FB2B882380ACE7C0462B000020A9
:105CB8009603002094030020A8030020600300201E
:105CC8005E0300205C03002070B58026A024802598
:105CD800E405760131002D0120000122FDF788FA44
:105CE800290001222000FDF783FA042000F094FC2B
:105CF800310000222000FDF77BFA042000F08CFC24
:105D0800290000222000FDF773FA70BD70B58026C7
:105D1800A0248025E405360131006D012000002211
:105D2800FDF766FA290000222000FDF761FA042039
:105D380000F072FC310020000122FDF759FA290019
:105D480001222000FDF754FA042000F065FC70BD24
:105D58008021A02070B501224901C005FDF748FA4D
:105D6800012000F059FC8021A02001220901C00572
:105D7800FDF73EFA8026012000F04EFC65257601ED
:105D8800A0203100C005FDF72DFA041E07D102003E
:105D98008021A0200901C005FDF72AFA06E0013D8F
:105DA800EDB2002DECD1FFF7B1FF0124200070BD4A
:105DB80070B58025A0248026E4052D0129007601F0
:105DC80020000022FDF714FA310000222000FDF720
:105DD8000FFA022000F020FC290001222000FDF724
:105DE80007FA022000F018FC290020000022FDF725
:105DF800FFF9310001222000FDF7FAF970BD70B5F6
:105E08008025A0248026E4052D01290076012000A4
:105E18000022FDF7EDF9310001222000FDF7E8F935
:105E2800042000F0F9FB290001222000FDF7E0F929
:105E3800042000F0F1FB290020000022FDF7D8F92A
:105E4800310001222000FDF7D3F970BDF8B580219B
:105E58000400A0200022A02680270901C005FDF724
:105E6800C7F90825F6053F0163B20122002B00DBC4
:105E78000022802130004901FDF7BAF9022000F024
:105E8800CBFB012239003000FDF7B2F9022000F007
:105E9800C3FB013D002239003000FDF7A9F9640079
:105EA8000220EDB200F0B8FBE4B2002DDCD1F8BD61
:105EB800F7B58027A0260825002401903F01F605A4
:105EC800002239003000FDF793F9022000F0A4FB0E
:105ED800390030000122FDF78BF980216400300081
:105EE8004901E4B2FDF77EF9002801D00134E4B29B
:105EF800013D0120EDB200F08FFB002DE0D1019BA8
:105F0800002B03D1FFF77BFF2000FEBDFFF750FFFA
:105F1800FAE70000F0B585B0FFF78EF8D14B1A8884
:105F2800D14B1A801A88002A03D01988CF4A914287
:105F380001D101221A80CE4B1A88CE4B1A801A88BA
:105F4800002A03D01988C94A914202D1AF2292008F
:105F58001A80C94C1B8822689BB25363C74B002226
:105F68009A5EC74B1A801A88002A03D01A8812B280
:105F7800013201D10A221A80C24B00229A5EC24B1A
:105F88001A801A88002A03D01A8812B2013201D165
:105F980000221A80BD4B00229A5EBD4B1A801A88D7
:105FA800002A03D01A8812B2013201D100221A80C5
:105FB800188800B2FFF70EFCB64B00229A5EB64B6B
:105FC8001A801A88002A03D01A8812B2013201D125
:105FD80028221A80B14B00229B5E5A1C92B2012AD9
:105FE80001D896235B00AE4A1380AE4B00229B5E1D
:105FF8005A1C92B2012A00D80023AB4A1380AB4B3B
:10600800019200229B5E5A1C92B2012A00D83C23BE
:10601800A74A200013800292FDF756FE00212000B7
:10602800FEF774F8A34C2000FEF736F92022A249A7
:106038002000FEF741FEFA22A049A148FCF7A4FB84
:10604800A02000222021C005FDF7D2F8322100202F
:1060580000F08CFAFA210120490000F087FA0320A9
:10606800984900F083FAFA210420890000F07EFAAA
:106078000A21052000F07AFA0620934900F076FA02
:106088000720904900F072FA0820904900F06EFA53
:10609800002000F095FA00280AD0894C2000FCF76F
:1060A80007FCFEF7E5FFFA2220008449FCF76CFBA9
:1060B800012000F085FA002850D08548FDF7ECF85B
:1060C80001218448FDF79AF8019B00241C5F631C9A
:1060D8009BB2012B42D9012C40D07F4B7F4D1888B1
:1060E80000B2FBF70BFB00227D4BFBF703F8E3172D
:1060F8000600E018584080B20F00FBF7FFFA0B00CB
:10610800020039003000FAF7DBFCFBF7BBFA80B27B
:10611800031C00B2DC3001DA724B1B881AB2DC2A8D
:1061280000DDDC232B80704B1B785AB2002B00D18A
:106138002A800022AB5EDA179B185340029A9BB262
:106148000021515E694A8B4200DB32E113886849BD
:1061580001339BB28B4200D92DE11380022000F05D
:106168002FFA002804D0A0200421C005FDF746F826
:10617800032000F025FA002802D002225A4B1A7098
:10618800042000F01DFA00280BD0022000F004FAC9
:10619800A02001220421C005FDF72AF80122554B51
:1061A8001A70052000F00CFA002810D0524C20007C
:1061B800FEF7CEFE6379022B09D1206BFAF724F99A
:1061C8004E4D2870606BFAF71FF94D4D2870062068
:1061D80000F0F6F9002801D0FFF70CFD072000F0C9
:1061E800EFF900282FD03D4B03930020185E0028BC
:1061F80029D0444A13780133DBB2182B00D9DCE0EC
:106208001370414C354D0022A35E00216A5E3F4E5B
:10621800D01711189A184140D01712184240D817B1
:106228001B18434089B29BB25B189A4200DB0FE10E
:106238001D2904D90023019A1380FFF74BF8012385
:1062480033702B882380082000F0BAF9002800D189
:10625800A5E02F4C08222F49200000F0FFF92E4915
:1062680008225BE0007800089E050020FFFF000080
:1062780002780008A20300206C01002004780008BE
:10628800A0030020067800089E0300200878000874
:106298009A0300200A780008280000200C780008DB
:1062A800260000200E7800089403002010780008CB
:1062B8002400002070020020E1050020AA0300202D
:1062C800F8000020881300007017000040771B00BA
:1062D8005C01002000040050A80300209603002061
:1062E80000805B40EC6700082B0000209203002030
:1062F800102700002A000020240300209803002013
:106308009903002003060020420000200206002016
:106318002E000020300000203A000020524800F0F3
:106328009DF9524B524E188803930023E15E00B248
:106338002081401A0023F75EC317C0185840642311
:106348005843CB17C9185940678289B2F9F770FFCB
:10635800132824DC0A23E55EAF4220D0029B0022EA
:106368009B5EAB421BDA039B3580188800B2FBF7B3
:10637800C5F900223F4BFAF7BDFE060028000F00C2
:10638800FBF7BCF90B00020039003000FAF798FB64
:10639800FBF778F9019BA5811880E5812582364CA9
:1063A8002378002B00D173E6FFF700FC002323704D
:1063B8006EE60023D1E66423CFE6002313702F4B4B
:1063C8000027DF5F381AC2178318642053405843E8
:1063D800FB17F918594089B2F9F7A0FE0A2832D8F4
:1063E800224E308800B2FBF789F90022214BFAF7D8
:1063F80081FE040038000D00FBF780F902000B0055
:1064080020002900FAF75CFBFBF73CF9019B04B27A
:1064180030881C8000B2FBF771F90022154BFAF79F
:1064280069FEE3170600E018584080B20F00FBF73A
:1064380065F90B00020039003000FAF741FBFBF761
:1064480021F9039B18800A4A0C4B12881A80D8E657
:106458003378012B06D11D2904D90023019A138012
:10646800FEF738FF0023EBE638000020A8030020E1
:106478009603002000805B400106002044000020B5
:10648800002370B50C251C0012492800584301331D
:106498000A1854609460547044540A2BF5D1FA21B8
:1064A8000D4B89001868F9F739FE802301385B0421
:1064B80098420DD2C021094A090650600848036A6B
:1064C8001B021B0A0B43036207239460136070BD11
:1064D800FEE7C0460C0600200000002010E000E0A7
:1064E80000ED00E01B4A70B51368002B07D0136855
:1064F800013B1360002B02D10122174B1A700022B6
:106508000C25012615482C00544303195968002905
:106518000AD0596801395960002905D15E70215C9B
:10652800012901D19968596001320A2AEBD10C4B33
:106538001A6801321A6019680A4A914201D1002288
:106548001A60094A13780133DBB2092B00D90023FA
:10655800137070BD88060020840600200C060020F9
:1065680008060020FFFFFF7F04060020020010B588
:10657800092800D9FEE7012484F310880C20504331
:10658800044B1A185160916000215170C45481F372
:10659800108810BD0C0600200300092800D9FEE76A
:1065A800012282F310880C2058430023034A111853
:1065B8004B604B70835483F3108870470C0600209F
:1065C80002000020092A09D80C214A43054B9B18D0
:1065D80059780022C8B2012901D15A7070471000B9
:1065E800FCE7C0460C06002000280FD0012800D187
:1065F8000130012383F310880022054B1860054BF6
:106608001A7082F310881A78012AFCD17047C046A4
:1066180088060020840600200D4B70B50D49060041
:106628001868F9F77BFD00230B4C46436568A168A1
:10663800A2689142FCD006D95B189B1AB34200D3DA
:1066480070BD1100F4E7A81AC318CB18F6E7C046C6
:106658000000002040420F0010E000E010B5884222
:1066680006D800239A4208D0CC5CC4540133F9E719
:106678008B189842F5D2013A00D210BD8B5C835436
:10668800F9E703008218934200D17047197001336B
:10669800F9E7000070B500260C4C0D4D641BA410E2
:1066A800A64209D1002600F023F80A4C0A4D641BC3
:1066B800A410A64205D170BDB300EB589847013627
:1066C800EEE7B300EB5898470136F2E7F0670008A9
:1066D800F0670008F4670008F0670008002310B5A9
:1066E8009A4200D110BDCC5CC4540133F8E70000D5
:1066F800F8B5C046F8BC08BC9E467047F8B5C04619
:10670800F8BC08BC9E46704701B40248844601BCE8
:08671800604700BF49000020AA
:10672000B00B0008A20B0008800B0008AC0B00089F
:10673000800B0008960E0008800B0008AC0B0008C8
:10674000A20B0008A20B0008960E0008AC0B000874
:10675000680B0008680B0008680B0008080F0008A9
:106760000000000000000000000000000000000029
:10677000010000000200000003000000040000000F
:106780000000000000000000000000000000000009
:1067900000000000000000000000000000000000F9
:1067A00001000000020000000300000004000000DF
:1067B00006000000070000000800000009000000BB
:1067C00004020800010002000400060008000A009C
:1067D0000C001000200040008000000108040204AA
:1067E00008010101010101030701000024FF00006D
:0467F000E1000008BC
:0467F400B9000008E0
:1067F8000024F40001000000040000000100FE0174
:1068080030024443452D323430362D56352E365F0E
:1068180048414C003C002C01280001010100010006
:10682800010001000100010000000000000000005C
:1068380000006E006E00000080220C4B30B55C69D1
:10684800D20222435A61EFF3108272B64C1CFF3415
:10685800401A0D68455004318C42FAD18021490212
:1068680018690842FCD182F3108830BD002002402C
:04000005080020854A
:00000001FF
